:020000040000FA
:100000002500050483061C0A58071D0A17020E0E58
:1000100037000600C80C02005804B609010CB000F5
:100020000307B10030024307190A31024307190AD6
:100030000008580506020300E409090C24006000CA
:10004000A40204021F0E43071F0A710C270066005A
:1000500076000E0C37000600C80C02007200730018
:10006000E409A809330AD3092607330A4607330AE5
:1000700072007300D3092607400A4607440A380A6B
:100080004607330A7805480A2607330A7804480ADF
:10009000D3097807500A2606380A4606480A550A40
:1000A0004606380A2606480A550AD309B20243060C
:1000B000B3022607550A4607550A050C3500D30931
:1000C000B2024306B3024306030078076A0A260613
:1000D0005D0A6D0A46065D0A6D0AF5025F0AD309DC
:1000E000B2024306B3024306030078077C0A2606E1
:1000F000030046066F0A810A4606030026066F0AB9
:10010000810AD3092607810A4607810A3302430779
:10011000900A1A0C92000306900A050C3200940A09
:10012000140CB2000307F300A8093805D9093804F4
:100130009E09E409AF09E009A809950A7807A30A0E
:1001400036043704A50A56045704170206000008AF
:100150003605560537055705170206000008360410
:100160005604370457041702060000083807C40A6B
:100170000602960157017807BF0A020EC00A040E54
:100180004306C40A1805C80A050C34001804C80A36
:100190001807CD0AF4004306CE0A00080E0C3700FB
:1001A000060058040300010C3000710058050602D7
:1001B000030012023000130231005805060203004A
:1001C000CA0C02000400E80ACC0C02000400E80A91
:0C01D000010C300071005805060203000D
:021FFE00EF0FE3
:00000001FF
